:10000000830100308A0004282030840031300D2024
:100010008301072904068001840A0406031D0A28B7
:1000200000348312BD00BE1B1C283E088A003D0818
:10003000BD0A0319BE0A820083133E1883173D08C8
:10004000BD0A84000008080082072834A0343B342D
:1001F4008312AA000430AB005330AC00AC0B0029CE
:10020400AB0BFE28AA0BFC280800073083129900C8
:10021400183083169F0010308500831285018D30BD
:100224009F0083121D21B9212208AA002108AB00D6
:1002340023085D2113298F3083129F009F182029E2
:100244001E08B400B30183161E08B100B2013308BE
:10025400B1070318B20A3408B207E823310883123D
:10026400A4003208A5003308A6002408B400250819
:10027400B5002608B600B101C830B2004230B30060
:1002840071230030BE0025301120B4001320B500C6
:100294001320B60071233108A7003208A8003308E0
:1002A400A9002708B1002808B2002908B300B22326
:1002B4003108A00008008312AC00AD01AE01AE0A03
:1002C400AF012C08B100B2012F083202031D6C29C2
:1002D4002E083102031805152C08B100B2012F08AD
:1002E4003202031D77292E083102031C05112A0846
:1002F400B100B2012F083202031D82292E083102F7
:10030400031885142A08B100B2012F083202031D14
:100314008D292E083102031C85102B08B100B2016F
:100324002F083202031D98292E08310203180514E0
:100334002B08B100B2012F083202031DA3292E0895
:100344003102031C05100330B000B00BA729AE0A1C
:100354000319AF0A01302F02003003192E02031CC7
:100364006329AD0A19302D020318080060291430DE
:10037400831220020318C229FF30A300A201A100A6
:10038400143020021530031CCF2920020318CE2973
:10039400FF30A300A201A100153020021630031C77
:1003A400DC2920020318DB29CC30A300A201FF3092
:1003B400A100163020021730031CE929200203187B
:1003C400E8299930A300A201FF30A10017302002D0
:1003D4001830031CF62920020318F5296630A300FF
:1003E400A201FF30A100183020021930031C032A97
:0C03F40020020318022A3330A300A201EB
:10040000FF30A100193020021A30031C0F2A2002ED
:1004100003180E2AA301A201FF30A1001A30200206
:100420001B30031C1C2A200203181B2AA301333093
:10043000A200FF30A1001B3020021C30031C292A1F
:1004400020020318282AA3016630A200FF30A10071
:100450001C3020021D30031C362A20020318352AC6
:10046000A3019930A200FF30A1001D3020021E30F0
:10047000031C432A20020318422AA301CC30A20005
:10048000FF30A1001E3020021F30031C4F2A200223
:1004900003184E2AA301FF30A200A1001F30200242
:1004A0002030031C5C2A200203185B2AA301FF30C2
:1004B000A200CC30A100203020022130031C692A88
:1004C00020020318682AA301FF30A2009930A1007E
:1004D000213020022230031C762A20020318752ABC
:1004E000A301FF30A2006630A10022302002233099
:1004F000031C832A20020318822AA301FF30A200D2
:100500003330A100233020022430031C8F2A200224
:1005100003188E2AA301FF30A200A101243020027B
:100520002530031C9C2A200203189B2A3330A30089
:10053000FF30A200A101253020022630031CA92A89
:1005400020020318A82A6630A300FF30A200A101F0
:10055000263020022730031CB62A20020318B52AB1
:100560009930A300FF30A200A101273020022830DB
:10057000031CC32A20020318C22ACC30A300FF3078
:10058000A200A101283020022930031CCF2A20021A
:100590000318CE2AFF30A300A200A10129302002B7
:1005A0002A30031CDC2A20020318DB2AFF30A300B8
:1005B000CC30A200A1012A3020022B30031CE92AF2
:1005C00020020318E82AFF30A3009930A200A101FD
:1005D0002B3020022C30031CF62A20020318F52AA7
:1005E000FF30A3006630A200A1012C3020022D3084
:1005F000031C032B20020318022BFF30A30033300F
:10060000A200A1012D3020022E30031C0F2B20024E
:1006100003180E2BFF30A300A201A1012E302002EF
:10062000031C0800FF30A300A201A10108008408F8
:1006300003190034330880008403320880008403E7
:10064000310880000034B901320D330DB70037088E
:1006500003192E2BB90DB301B2170800B101B20175
:10066000B3010034B910350D360DB8003808031940
:100670003E2B0318B914B601B5170800B801B40130
:10068000B501B6010800370803192E2BB213B90CB7
:10069000370CB3000318B217172BB708031D612BD3
:1006A000B101B201B301172B33030319B10A0319C6
:1006B000B20A0319B30A0310B30CB20CB10CB70A97
:1006C0004D2BB308031D542B310832040319502B52
:1006D000B21B432BB7030319502B0310B10DB20DFE
:1006E000682B840123233223BA01BB01BC010730EC
:1006F000B6000310B50CB40C031C892B3108BA07E3
:1007000032080318320FBB0733080318330FBC0736
:100710000310B10DB20DB30DB60B792B0930B60035
:10072000952B0310BC0CBB0CBA0C0310B50CB40C0D
:10073000031CA42B3108BA0732080318320FBB0779
:1007400033080318330FBC07B60B912B7A303807E8
:10075000B707390CB9063A08B1003B08B2003C08AB
:10076000B3004D2B84012323B4018230B707B71B9C
:100770002E2BF030B707B71BCE2B183037020318DB
:100780002E2BB708031DC72B3918F1230800B70318
:100790000310B10DB20DB30DB40DC12B0310B30C8A
:1007A000B20CB10CB70FCE2BC42BB41FDA2B3914FB
:1007B000F123DB2BB9018E30B7008401B408031993
:1007C0004D2B0310B40CB30CB20CB10CB70ADE2BDA
:1007D000B301B21BB3033308B400D52BB301B4018A
:1007E000DA2B0310FF30B107B109031CB207B209BD
:0E07F000031CB307B309031CB407B4090800C7
:02400E00C43FAD
:00000001FF
